:020000020000FC
:10000000024A4B02470E00000000000245AB000010
:10001000000000024F540000000000023BB300004B
:10002000000000023685C2AF758F0153A2DFD29364
:10003000C200124B6D124BE8125486122E55E4F595
:100040002274042522F582E43460F583E0FF74F81D
:100050002522F582E4347FF583EFF00522E522B412
:1000600006DF90602BE024FF920A90602FE0600C86
:10007000E064016007E4FD7F2C12512D906031E0B7
:10008000F46003E07004C2078009906031E0B401BD
:1000900002D207906020E09060A5F0906021E0908F
:1000A00060AAF09060A5E0FFB408089060AAE06440
:1000B00001600BEFB4080C9060AAE0B40205752350
:1000C00003800375230190601FE0FFAD2312486792
:1000D0001254E6E49060A8F0A3F09060A6F0A3F0BC
:1000E000D2AF9060BA7407F0A374D0F0200A0C7BF2
:1000F000FF7A4379B9125357124CB91254369060B3
:1001000023E0B40203439040124D131255391253A9
:100110003290602EE024FF920430040B12505712EC
:100120003F6E122E558003125091C28AD2AA90605F
:1001300017E0FFA3E09060B8CFF0A3EFF0E4F52262
:1001400074132522F582E43460F583E0FF74C5253D
:1001500022F582E43460F583EFF00522E522B40451
:10016000DF200A097BFF7A4379CF125357756680E7
:100170007BB47A057D02E4FF12490A7566807BB57F
:100180007A057D017F0312490A7F0312546D200A0C
:10019000097BFF7A4379E4125504300406300803E2
:1001A0001219FA12443B30061A7D017F02122447CD
:1001B000906066E0B5060AA3E0B507057F0212313C
:1001C00071C20690602FE06401600D90600AE064E7
:1001D000016005E0640270433002409060A4744105
:1001E000F09060B9E02401FB9060B8E03400FA754B
:1001F00066807D027F0112490A75430075440175CE
:1002000045017546607547C57548007549077B010E
:100210007A6079A47F01124127C2029060ABE0703E
:100220000D1228C57F057E001252E602019A9060E9
:10023000ACE06401706430090302049B7D027F021C
:100240001224478E248F25D3EF9400EE648094808F
:100250004009AD25AC247F02123CAC1216F9906027
:10026000CBEEF0A3EFF04E7018906023E0B40111D4
:10027000E518B4010CC2AF7F111250C6D2AFE4F53D
:10028000189060CBE0FEA3E0FFD39400EE94005002
:100290000302019A1247BC02019A9060AEE0640129
:1002A000600302034D9060ADE0600302034D906077
:1002B000A6E0FEA3E0FFA3E06E7003A3E06F70036F
:1002C00002034D9060BAE475F001120572ABF0FACA
:1002D0007566807D017F0212490ABFFF18C39060D6
:1002E000BBE094FF9060BAE094FF40D77407F0A39E
:1002F00074D0F080CE7B017A60791990601DE0F5B2
:100300002CA3E0F52D7F021242B8EFF4602E90602E
:10031000AB7401F09060ADF0E4A3F0C2929060ADD8
:10032000E0906030F0C2AFE49060B6F09060A2F070
:10033000A3F09060C1F0A3F0D2AF8011C2AF906083
:10034000A6E0FFA3E0A3CFF0A3EFF0D2AFE4FD7FE0
:10035000021224479060B5EFF0700302047124F993
:10036000700302043704600302019A9060AEE0FF5C
:1003700064016005EF6402703B9060ADE07035048D
:10038000F0C292906030F0C2AFE49060B6F090603E
:10039000A2F0A3F09060C1F0A3F09060A8F0A3F0E9
:1003A0009060A6F0A3F0D2AF200A097BFF7A4379D0
:1003B000E91255047D027F021224478E248F25D333
:1003C000EF9400EE648094804023D3E5259400E50B
:1003D00024648094885016E4FD7F02122447EF6461
:1003E000064E7009AD25AC247F02123CAC1216F902
:1003F0009060CBEEF0A3EFF04E7018906023E0B465
:100400000111E518B4010CC2AF7F111250C6D2AF72
:10041000E4F5189060CBE0FEA3E0FFD39400EE94E7
:100420000040031247BC9060B6E0700302019A7F5F
:1004300002124E1702019A7D027F021224478E2477
:100440008F25D3EF9400EE64809480401CD3E52583
:100450009400E5246480948840067524087525007E
:10046000AD25AC247F02123CAC7F02124E17020174
:100470009A7F02124E17E49060ADF09060ABF0D21C
:10048000929060ADE0906030F0300A0302019A7BF8
:10049000FF7A4379F512550402019A200A097BFF7D
:1004A0007A4479021255047F02124E170200FE228E
:1004B000BB010689828A83E0225002E722BBFE024A
:1004C000E32289828A83E49322BB010CE58229F529
:1004D00082E5833AF583E0225006E92582F8E62298
:1004E000BBFE06E92582F8E222E58229F582E58352
:1004F0003AF583E49322BB010689828A83F0225075
:1005000002F722BBFE01F322F8BB010DE58229F5BB
:1005100082E5833AF583E8F0225006E92582C8F6A1
:1005200022BBFE05E92582C8F222EF8DF0A4A8F0D7
:10053000CF8CF0A428CE8DF0A42EFE22C2D5EC30B4
:10054000E709B2D5E4C39DFDE49CFCEE30E715B2AB
:10055000D5E4C39FFFE49EFE120834C3E49DFDE48E
:100560009CFC800312083430D507C3E49FFFE49E4F
:10057000FE22A3F8E0C5F025F0F0E58215827002B6
:100580001583E0C838F0E822BB010A89828A83E03B
:10059000F5F0A3E022500687F009E71922BBFE0719
:1005A000E3F5F009E3192289828A83E493F5F07474
:1005B000019322BB010A89828A83F0E5F0A3F0222D
:1005C0005006F709A7F01922BBFE06F3E5F009F380
:1005D000192275F008758200EF2FFFEE33FECD3340
:1005E000CDCC33CCC58233C5829BED9AEC99E582A4
:1005F00098400CF582EE9BFEED9AFDEC99FC0FD530
:10060000F0D6E4CEFBE4CDFAE4CCF9A88222B8001F
:10061000C1B90059BA002DEC8BF084CFCECDFCE5EA
:10062000F0CBF97818EF2FFFEE33FEED33FDEC330E
:10063000FCEB33FB10D703994004EB99FB0FD8E593
:10064000E4F9FA227818EF2FFFEE33FEED33FDECDC
:1006500033FCC933C910D7059BE99A4007EC9BFCD2
:10066000E99AF90FD8E0E4C9FAE4CCFB2275F0105E
:10067000EF2FFFEE33FEED33FDCC33CCC833C81083
:10068000D7079BEC9AE899400AED9BFDEC9AFCE8B1
:1006900099F80FD5F0DAE4CDFBE4CCFAE4C8F922FE
:1006A000C3E49FFFE49EFEE49DFDE49CFC22EB9FDF
:1006B000F5F0EA9E42F0E99D42F0E89C45F022BB4D
:1006C000010789828A830208955005E9F8020889A2
:1006D000BBFE05E9F80208A189828A830208ADEC15
:1006E000F0A3EDF0A3EEF0A3EFF022A8828583F053
:1006F000D083D082120702120702120702120702E9
:10070000E473E493A3C583C5F0C583C8C582C8F06C
:10071000A3C583C5F0C583C8C582C822D083D08253
:10072000F8E4937012740193700DA3A393F874010D
:1007300093F5828883E4737402936860EFA3A3A3A4
:1007400080DFE709F608DFFA8046E709F208DFFAFA
:10075000803E88828C83E709F0A3DFFA8032E309C8
:10076000F608DFFA8076E309F208DFFA806E888205
:100770008C83E309F0A3DFFA806289828A83E0A395
:10078000F608DFFA805689828A83E0A3F208DFFA4E
:10079000804A80D280FA80C680D4806580F2803121
:1007A000801080A680EA809A80A880DA80E280CAE1
:1007B000803189828A8363A20188828C8363A2014B
:1007C000E493A363A201F0A363A201DFF3DEF1804F
:1007D0000B89828A83E493A3F608DFF9ECFAA9F087
:1007E000EDFB2289828A8363A20188828C8363A2C3
:1007F00001E0A363A201F0A363A201DFF4DEF280B3
:10080000DB89828A83E493A3F208DFF980CE88F043
:10081000EF60010E4E60C588F0ED2402B404005074
:10082000BBF582EB2402B4040050B123234582239C
:1008300090079273BC000BBE0029EF8DF084FFADD2
:10084000F022E4CCF875F008EF2FFFEE33FEEC3326
:10085000FCEE9DEC984005FCEE9DFE0FD5F0E9E422
:10086000CEFD22EDF8F5F0EE8420D21CFEADF07541
:10087000F008EF2FFFED33FD4007985006D5F0F25A
:1008800022C398FD0FD5F0EA22E6FC08E6FD08E653
:10089000FE08E6FF22E0FCA3E0FDA3E0FEA3E0FFEC
:1008A00022E2FC08E2FD08E2FE08E2FF22E493FCFB
:1008B000740193FD740293FE740393FF228F388CAE
:1008C000398D3A8A3B8B3CE4FDAF38122447EF4E1A
:1008D00070057EFF7FFF22C2A8E53875F003A424CF
:1008E000E0FFE5F034818F82F583E0F5567F027EEC
:1008F000001254B2E53875F00CA4FFAEF02410FDE0
:10090000EE34808D82F583E0F54AA3E0F54BEF24C9
:1009100010FFEE3480FE8F82F583A3A3E0F54C8FA9
:10092000828E83A3A3A3E0F54DE53875F003A424DC
:10093000E1FFE5F034818F82F583E0F5567F027E9A
:10094000001254B2E53875F00CA4FFAEF02414FD8B
:10095000EE34808D82F583E0F54EA3E0F54FEF2471
:1009600014FFEE3480FE8F82F583A3A3E0F5508F51
:10097000828E83A3A3A3E0F551D2A8D3E53C9400D3
:10098000E53B94005004E4FEFF22AF51AE50AD4F62
:10099000AC4EAB4DAA4CA94BA84AC31206AE401AA6
:1009A000E54D9551F555E54C9550F554E54B954F72
:1009B000F553E54A954EF552801FAF51AE50AD4FFD
:1009C000AC4E1206A0EF254DF555EE354CF554ED25
:1009D000354BF553EC354AF552E53825E0245AF508
:1009E00082E43460F583E0FEA3E0FFC3953CEE951E
:1009F0003B50048E3B8F3CAE3BAF3CE4FCFDAB5523
:100A0000AA54A953A852C31206AE50227F017E00F9
:100A100012530CE53875F018A424A1FFE5F03480DA
:100A20008F82F583E05407640270030208C7E5383B
:100A300025E02408F8E6FA08E6FBE53825E025E09D
:100A4000243AF582E43460F583E0FCA3E0FDA3E002
:100A5000FEA3E05551FFEE5550FEED554FEC554EBF
:100A6000EF2BFFEE3AA907754701F5488949E538AC
:100A700075F018A424A1FFE5F034808F82F583E09F
:100A8000540764026003020C6CAC48AD017A607BD1
:100A9000D3F55C755D08AF381239B79060D5E0AB1F
:100AA0003DAA3EA93F1204F69060D6E0AB3DAA3EB7
:100AB000A93F9000011205089060D7E09000021253
:100AC00005089060D8E09000031205089060D9E016
:100AD000FFAB40AA41A942E48FF01205B3AB40AA94
:100AE00041A942120588FE9060DAE07C002400FFF4
:100AF000EC3E8FF01205B3E4F543F544F545F546B9
:100B0000D3E53C9400E53B94005003020C6C9060EC
:100B1000D4E024F8FF9060D3E034FFFEE48F558EDC
:100B200054F553F552E5512408F551E43550F5508C
:100B3000E4354FF54FE4354EF54EE53825E0240811
:100B4000F8E6FA08E6FBE53825E025E0243AF582E8
:100B5000E43460F583E0FCA3E0FDA3E0FEA3E055F0
:100B600051FFEE5550FEED554FEC554EEF2BFFEE7D
:100B70003AA907754701F5488949FCAD01E53A25D1
:100B800044FBE5393543FA85545C85555DAF381231
:100B900039B78E458F46E4FCFDE5512FF551E55000
:100BA0003EF550ED354FF54FEC354EF54EE546250B
:100BB00044F544E5453543F543E5552408FDE43562
:100BC00054FCC3E53C9DFFE53B9CFEF53B8F3CD3CD
:100BD000EF9400EE94005003020B00E53825E0246A
:100BE00008F8E6FA08E6FBE53825E025E0243AF5C2
:100BF00082E43460F583E0FCA3E0FDA3E0FEA3E023
:100C00005551FFEE5550FEED554FEC554EEF2BFF75
:100C1000EE3AA907754701F5488949FCAD017A60AC
:100C20007BD3755C00755D08AF381239B7AB40AA4D
:100C300041A942120588FF9060D9E0FCA3E0FDB510
:100C4000072AECB5F026ED64434C6020AB3DAA3E8C
:100C5000A93F1206BF9060D5E0F8A3E0F9A3E0FA3F
:100C6000A3E0FBC31206AE7003020B00E53875F07B
:100C70000CA42414FFE5F03480FE8F82F583E54E4A
:100C8000F0A3E54FF08F828E83A3A3E550F08F820F
:100C90008E83A3A3A3E551F0E42538FFE434808FCD
:100CA00082F5837440F0AE43AF44228F2A8C2B8DA3
:100CB0002CE4F52DF52EF52FF530F531F537F53619
:100CC00074322536F582E4347BF58374FFF0053603
:100CD000E536B408EBE52A70237C7B7D00F53D7595
:100CE0003E00753F32F54075410075422DAB2CAA90
:100CF0002BAF2A1208BD8E2F8F30801BE52AB4033C
:100D0000167C7B7D00AB2CAA2BFF122C8B8E2F8F99
:100D100030752D13752E89E52E64897004E52D64D8
:100D200013600302107C200A097BFF7A4D796A1256
:100D30005504907B00E064467079A3E064497073C9
:100D4000A3E0644E706DA3E0644470677A7B790021
:100D500078007C7B7D017B017A607900FE7F3A120E
:100D6000080E907B007449F0A3744DF0A37449F011
:100D7000A3744EF07532FF7533FF7534FF7535FF80
:100D8000752D13752E8975430075443275450075B0
:100D90004600754732852D48852E497B017A7B793F
:100DA00000AF2A1241277F017E001252E675310101
:100DB00002107C907B00E064536003020FEBA3E021
:100DC00064456003020FEBA3E064546003020FEB81
:100DD000A3E064546003020FEB907FF8E0FF907B88
:100DE00004E06F600302107C907FF9E0FF907B05C8
:100DF000E06F600302107C907FFAE0FF907B06E0DA
:100E00006F600302107C907FFBE0FF907B07E06F38
:100E1000600302107C907FFCE0FF907B08E06F6035
:100E20000302107C907FFDE0FF907B09E06F600380
:100E300002107C200703020F83F53674322536F545
:100E400082E43460F583E0FF74E62536F582E4340D
:100E500060F583EFF00536E536B408DF9060E6E034
:100E6000FF907B32E06F70599060E7E0FF907B333A
:100E7000E06F704D9060E8E0FF907B34E06F704170
:100E80009060E9E0FF907B35E06F70359060EAE0BC
:100E9000FF907B36E06F70299060EBE0FF907B372E
:100EA000E0B5071D9060ECE0FF907B38E0B50711DE
:100EB0009060EDE0FF907B39E0B507057537018064
:100EC00003E4F537E53764017068907B007453F0F4
:100ED000A37445F0A37454F0A37443F0752D1375F7
:100EE0002E897532FF7533FF7534FF7535FF7543F5
:100EF00000754432754500754600754732852D48AA
:100F0000852E497B017A7B7900AF2A1241277F0128
:100F10007E001252E67A60790078007C607D017B69
:100F2000017A7B79007E007F3A12080E7531020249
:100F3000107C907B007446F0A37441F0A37449F0D8
:100F4000A3744CF0752D13752E897532FF7533FF20
:100F50007534FF7535FF754300754432754500756E
:100F60004600754732852D48852E497B017A7B796D
:100F700000AF2A1241277F017E001252E6E4F531CC
:100F800002107C907B007453F0A37445F0A374545A
:100F9000F0A37443F0752D13752E897532FF7533E8
:100FA000FF7534FF7535FF75430075443275450094
:100FB000754600754732852D48852E497B017A7B21
:100FC0007900AF2A1241277F017E001252E67A6033
:100FD000790078007C607D017B017A7B79007E005E
:100FE0007F3A12080E75310202107C907B00E0649B
:100FF00046600302107CA3E06449600302107CA3F6
:10100000E064527077A3E064537071907FF8E0FF62
:10101000907B04E06F7065907FF9E0FF907B05E0C6
:101020006F7059907FFAE0FF907B06E06F704D90F3
:101030007FFBE0FF907B07E06F7041907FFCE0FF5B
:10104000907B08E06F7035907FFDE0FF907B09E0BA
:101050006F7029121CAFEF64014E7011200A097BDA
:10106000FF7A4D797E12535712501B800F200A09C8
:101070007BFF7A4D79871255047F0022AF3122AB76
:1010800005A907E4F538F539F53AF53B908096E97E
:10109000F0908095EBF07510C07511007508E07543
:1010A0000900E4FAEAFD3395E0FCED25E0FFEC33BE
:1010B000FE74622FF58274603EF583E4F0A3F07451
:1010C0005A2FF58274603EF583E4F0A3F0C3E5384F
:1010D000648094A040030211E4EA25E0FFE9A80738
:1010E000088002C313D8FC5403146049147003022F
:1010F00011701470030211AB240360030211E4EDBC
:1011000025E0FFEC33FE74622FF58274603EF583B8
:101110007404F0A3E4F0EDAE047802C333CE33CE12
:10112000D8F9244AF58274603EF5831206EB00007C
:1011300003FF0211E4EAFD3395E0FCED25E0FFEC4E
:1011400033FE74622FF58274603EF5837408F0A359
:10115000E4F0EDAE047802C333CE33CED8F9244A9E
:10116000F58274603EF5831206EB000007FF807481
:10117000EAFD3395E0FCED25E0FFEC33FE74622FD1
:10118000F58274603EF5837410F0A3E4F0EDAE04D4
:101190007802C333CE33CED8F9244AF58274603E48
:1011A000F5831206EB00000FFF8039EAFD3395E06E
:1011B000FCED25E0FFEC33FE74622FF58274603E97
:1011C000F5837420F0A3E4F0EDAE047802C333CECF
:1011D00033CED8F9244AF58274603EF5831206EBCB
:1011E00000001FFFC3E53A648094A040030213018E
:1011F000EA25E0FFEBA807088002C313D8FC5403DC
:1012000014604F14700302128D1470030212C8246C
:10121000036003021301EAFD3395E0FCED25E0FFD6
:10122000EC33FE745A2FF58274603EF5837404F03B
:10123000A3E4F0EDAE047802C333CE33CED8F92464
:101240003AF58274603EF5831206EB000003FF025C
:101250001301EAFD3395E0FCED25E0FFEC33FE746D
:101260005A2FF58274603EF5837408F0A3E4F0ED24
:10127000AE047802C333CE33CED8F9243AF5827463
:10128000603EF5831206EB000007FF8074EAFD3331
:1012900095E0FCED25E0FFEC33FE745A2FF58274E7
:1012A000603EF5837410F0A3E4F0EDAE047802C361
:1012B00033CE33CED8F9243AF58274603EF58312EA
:1012C00006EB00000FFF8039EAFD3395E0FCED25C9
:1012D000E0FFEC33FE745A2FF58274603EF58374A0
:1012E00020F0A3E4F0EDAE047802C333CE33CED8C1
:1012F000F9243AF58274603EF5831206EB00001F74
:10130000FFEAFF3395E0FEEF25E0FFEE33FE746267
:101310002FF58274603EF583E0FCA3E02539F539B2
:10132000EC3538F538745A2FF58274603EF583E059
:10133000FEA3E0253BF53BEE353AF53AEA606B2536
:10134000E0240EF8E6FC08E6FDEAFF3395E0FEEF48
:1013500025E0FFEE33FE74602FF58274603EF58366
:10136000E0FEA3E02DFFEE3CFEEA25E02410F8A607
:101370000608A607EA25E02406F8E6FC08E6FDEAEA
:10138000FF3395E0FEEF25E0FFEE33FE74582FF5B6
:101390008274603EF583E0FEA3E02DFFEE3CFEEAA2
:1013A00025E02408F8A60608A6070AEA64046003F4
:1013B0000210A4E490606AF090800004F090606AEB
:1013C000E030E0F9228F4C8B4D8A4E894FC2A8E560
:1013D0004C75F003A424F0FFE5F034818F82F5838F
:1013E000E0F5527F027E001254B2E54C75F00CA479
:1013F000FFAEF02440FDEE34808D82F583E0F5559C
:10140000A3E0F556EF2440FFEE3480FE8F82F58393
:10141000A3A3E0F5578F828E83A3A3A3E0F558E53D
:101420004C75F003A424F1FFE5F034818F82F5833D
:10143000E0F5527F027E001254B2E54C75F00CA428
:10144000FFAEF02444FDEE34808D82F583E0F55943
:10145000A3E0F55AEF2444FFEE3480FE8F82F5833B
:10146000A3A3E0F55B8F828E83A3A3A3E0F55CD2F8
:10147000A8AF5CAE5BAD5AAC59AB58AA57A956A8F9
:1014800055C31206AE4029AE5BAF5CAC57AD58ED0C
:101490009FFFEC9EFEE54C25E02462F582E434607B
:1014A000F583E0FCA3E0C39FF554EC9EF553802E3A
:1014B000AE5BAF5CC3E49FFFE49EFEAC57AD58EF5C
:1014C0002DFFEE3CFEE54C25E02462F582E434601D
:1014D000F583E0FCA3E0C39FF554EC9EF553E54C87
:1014E00025E02462F582E43460F583E0FEA3E0C3E6
:1014F0009554EE9553500A7F017E0012530C02134F
:10150000CDE554455370097F01FE12530C0213CDF3
:10151000C3E5549551E55395505006855350855475
:1015200051E54C25E02410F8E6FA08E6FBE54C25E9
:10153000E025E0244AF582E43460F583E0FCA3E092
:10154000FDA3E0FEA3E05558FFEE5557FEED5556BE
:10155000EC5555EF2BFFEE3AA907755D01F55E8955
:101560005FAC4EAD4FFAAB01855067855168AF4C0B
:10157000123AB6AE50E4FCFDE5582551F558E55752
:101580003EF557ED3556F556EC3555F555E54C75A8
:10159000F00CA42440FFE5F03480FE8F82F583E553
:1015A00055F0A3E556F08F828E83A3A3E557F08F05
:1015B000828E83A3A3A3E558F07F027E001254B26B
:1015C000E4254CFFE434808F82F5837420F0E4F549
:1015D00053F554E4254CFFE434808F82F583E020FA
:1015E000E5030216747F017E0012530C0554E55486
:1015F000AE537002055314D394E8EE940340D4E53F
:101600004C75F00CA42444FFE5F03480FE8F82F585
:1016100083E555F0A3E556F08F828E83A3A3E557AB
:10162000F08F828E83A3A3A3E558F0AF4C124E1720
:10163000E54C75F018A4FDACF024AEFBEC34808BC7
:1016400082F583E0756100F560A3E02561F561E452
:101650003560F560ED24A1FFEC34808F82F583E0E6
:1016600054F0F566AB61AA607D02AF4C12490A7E68
:10167000FF7FFF22E4FDAF4C122447EF4E7075E56B
:101680004C75F00CA42444FFE5F03480FE8F82F505
:1016900083E555F0A3E556F08F828E83A3A3E5572B
:1016A000F08F828E83A3A3A3E558F0AF4C124E17A0
:1016B000E54C75F018A4FDACF024AEFBEC34808B47
:1016C00082F583E0756100F560A3E02561F561E4D2
:1016D0003560F560ED24A1FFEC34808F82F583E066
:1016E00054F0F566AB61AA607D02AF4C12490A7EE8
:1016F000FF7FFF22AE50AF5122E49060D3F0A3F001
:10170000C2AF9060A8E0FEA3E0FF9060CDEEF0A332
:10171000EFF09060A6E0FCA3E0FD9060CFECF0A3BA
:10172000EDF0D2AFEFB50508EEB50404E4FEFF22FC
:10173000906024E060030217EAA3E0FEA3E04E609D
:10174000030217EA906027E0FEA3E04E6003021751
:10175000EA9060CFE0FCA3E0FD9060CDE0FEA3E066
:10176000FFD39DEE9C4023EF9DFFEE9CFE9060D347
:10177000F0A3EFF074002DF9746B3CFA7B01780054
:101780007C737D0112080E0219F19060CFE0FAA37C
:10179000E0FBC3E49BFF74089AFEA3F0A3EFF09074
:1017A00060CDE0FCA3E02FFDEC3E9060D3F0A3ED14
:1017B000F074002BF9746B3AFA7B0178007C737D2E
:1017C0000112080E9060CDE0FEA3E0FF9060D1E032
:1017D000FCA3E02400F974733CA801FC7D017B01AB
:1017E0007A6B790012080E0219F1300B0F9060C36A
:1017F000E0FFA3E09060CDCFF0A3EFF09060CFE0EA
:10180000FEA3E0FF9060CDE0FCA3E0FDD39FEC9E43
:1018100050030218A3ED9FFFEC9E9060D3F0A3EF5E
:10182000F0200B03300C2A9060D3E0FEA3E0FF9081
:1018300060CFE0FCA3E02400F9746B3CFA7B0178F4
:10184000007C737D0112080E9060D3E0FEA3E0FFE0
:1018500022906025E0FEA3E0FF9060D3E0FCA3E0CF
:10186000C39FEC9E4033906025E0FFA3E09060D3DF
:10187000CFF0A3EFF09060D3E0FEA3E0FF9060CF45
:10188000E0FCA3E02400F9746B3CFA7B0178007C57
:10189000737D0112080E0219F1E49060D3F0A3F0F9
:1018A0000219F19060CFE0FEA3E0FFC3E49FFF7454
:1018B000089EFEA3F0A3EFF09060CDE0FCA3E02F24
:1018C000FFEC3E9060D3F0A3EFF0200B03300C4D03
:1018D0009060D1E0FEA3E0FF9060CFE0FCA3E024A5
:1018E00000F9746B3CFA7B0178007C737D0112086F
:1018F0000E9060CDE0FEA3E0FF9060D1E0FCA3E09D
:101900002400F974733CA801FC7D017B017A6B799A
:101910000012080E9060D3E0FEA3E0FF2290602545
:10192000E0FEA3E0FF9060D1E0FCA3E0C39FEC9E4B
:101930004041906025E0FFA3E09060D1CFF0A3EF9D
:10194000F0906025E0FFA3E09060D3CFF0A3EFF02C
:101950009060D1E0FEA3E0FF9060CFE0FCA3E02424
:1019600000F9746B3CFA7B0178007C737D011208EE
:101970000E807E906025E0FEA3E0FF9060D3E0FC47
:10198000A3E0C39FEC9E40629060D1E0FEA3E0FF25
:101990009060CFE0FCA3E02400F9746B3CFA7B017B
:1019A00078007C737D0112080E9060D1E0FEA3E008
:1019B000FF906025E0FCA3E0C39FFFEC9EFE9060DB
:1019C000D1E0FCA3E02400F974733CA801FC7D0184
:1019D0007B017A6B790012080E906025E0FFA3E08E
:1019E0009060D3CFF0A3EFF08007E49060D3F0A332
:1019F000F09060D3E0FEA3E0FF22E4F5287D027FB3
:101A000001122447AD07AC06D3ED9400EC940040DE
:101A1000077F01121F558F28906078E024FE602810
:101A2000147003021B25147003021BFE24036003C1
:101A3000021CAEE528B4020C7F0112269590607856
:101A40007402F0221238B322E52864056003021AFA
:101A5000E8123E87EF60381235549060787403F0D6
:101A600090609C1206EB0000000090609CE0FCA3DC
:101A7000E0FDA3E0FEA3E02405FFE43EFEE43DFD1F
:101A8000E43CFC9060871206DFE4906085F02290D1
:101A90006093E0FCA3E0FDA3E0FEA3E0FFE4FAF91D
:101AA000F8EF2401FFEA3EFEE93DFDE83CFC9060D2
:101AB000931206DF90609C1206EB0000000090601D
:101AC0009CE0FCA3E0FDA3E0FEA3E02405FFE43ED0
:101AD000FEE43DFDE43CFC9060871206DFE490608C
:101AE00085F090607804F022E528B4063490609C7C
:101AF0001206EB0000000090609CE0FCA3E0FDA358
:101B0000E0FEA3E02405FFE43EFEE43DFDE43CFCF2
:101B10009060871206DFE4906085F090607804F0B2
:101B2000221238B32274FFFFFEFDFC906074E0F8CF
:101B3000A3E0F9A3E0FAA3E0FBC31206AE70030230
:101B40001CAEE47B02FAF9F8906074E0FCA3E0FDBF
:101B5000A3E0FEA3E0FF12060E90609CE0F8A3E075
:101B6000F9A3E0FAA3E0FBD31206AE5003021CAEC9
:101B7000E4F528F527747D2527F582E43460F583A4
:101B8000E0FF74792527F582E43460F583EFF005F2
:101B900027E527B404DF7566807B447A007D027FE9
:101BA0000112490A906093E0FCA3E0FDA3E0FEA3CC
:101BB000E0FFE4FAF9F8EF2401FFEA3EFEE93DFD1B
:101BC000E83CFC9060931206DF7F0112269590603E
:101BD000787404F090609C1206EB000000009060A6
:101BE0009CE0FCA3E0FDA3E0FEA3E02405FFE43EAF
:101BF000FEE43DFDE43CFC9060871206DF22E52810
:101C00006405706E906085F0FFF527747D2527F5DB
:101C100082E43460F583E0FE74792527F582E434AC
:101C200060F583E06E60047F0180070527E527B437
:101C300004D9EF600D90609C1206EB0000000012CA
:101C4000355490609C1206EB0000000090609CE010
:101C5000FCA3E0FDA3E0FEA3E02405FFE43EFEE4D8
:101C60003DFDE43CFC9060871206DF9060787403D1
:101C7000F022E528B4063490609C1206EB000000C8
:101C80000090609CE0FCA3E0FDA3E0FEA3E024053F
:101C9000FFE43EFEE43DFDE43CFC9060871206DF7D
:101CA000E4906085F090607804F0221238B322C28C
:101CB0000DE49060E0F0A3F09060E4F0A3F0200A5F
:101CC000097BFF7A4D799712535712509143900434
:101CD000E4F5667BBE7A057D01FF12490AE4FF1236
:101CE000546DE4FDFF1224479060CFEFF0BF06175C
:101CF0009060D21206EB00000000E49060D6F0A3E2
:101D0000F0A3F0A3F080349060E5E004F07006905A
:101D100060E4E004F07F017E001252E6D39060E5BB
:101D2000E094C89060E4E0940040B7200A097BFF8B
:101D30007A4D79A6125357E4FEFF22E4FDFF1224E8
:101D4000479060CFEFF0BF06F2200D777D02E4FFF1
:101D5000122447C3EF940AEE940040DF7C607DD2EA
:101D60007B047A00E4FF122C8B7C607DDA7B067AA0
:101D700000E4FF122C8B9060DAE064576004E4FE0C
:101D8000FF229060DBE064696004E4FEFF22906063
:101D9000DCE0647A6004E4FEFF229060DDE0646EC3
:101DA0006004E4FEFF229060DEE064656004E4FE0F
:101DB000FF229060DFE064746004E4FEFF22D20D35
:101DC000021D3B7D02E4FF1224479060CDEEF0A39C
:101DD000EFF0D39400EE648094805003021D3B7CAE
:101DE000637D009060CDE0FAA3E0FBE4FF122C8B52
:101DF0009060CDEEF0A3EFF0E49060D0F0A3F0900F
:101E000060CDE0FEA3E0FF9060D0E0FCA3E0FDC366
:101E10009FEC9E502D74002DF58274633CF583E099
:101E2000FD9060D6E475F00112057285F082F583AD
:101E3000EDF09060D1E004F070069060D0E004F026
:101E400080BD9060E1E02FF09060E0E03EF09060B7
:101E5000D4E0FEA3E024FAFFEE34FFFE9060E0E061
:101E60006E7003A3E06F6003021D3B9060D6F0A389
:101E7000F09060D0F0A3F09060D2E0FCA3E0FDA36E
:101E8000E0FEA3E024F8FBEE34FFFAED34FFF9ECBA
:101E900034FFF89060D0E0FEA3E0FFE4FCFDD31235
:101EA00006AE402E9060D6E475F00112057285F002
:101EB00082F583E0FF9060D9E02FF09060D8E034A5
:101EC00000F09060D1E004F070069060D0E004F083
:101ED00080A59060D6E475F00112057285F082F558
:101EE00083E09060E2F09060D6E475F00112057234
:101EF00085F082F583E09060E3F09060D8E0A3FF86
:101F00009060E2E0FEEF6E6004E4FEFF229060D994
:101F1000E0FF9060E3E0FEEF6E6004E4FEFF22204D
:101F20000A147BFF7A4D79B21253579060D8E0FEC5
:101F3000A3E0FF1254D69080007410F09060D4E0BB
:101F4000FEA3E024F8FFEE34FF907FFEF0A3EFF055
:101F50007E007F0122AB05AA047C7D7D00753D00DB
:101F6000753E00753F2975400075410075422D1280
:101F700008BDAD07AC06E52E6443452D7070F53005
:101F800074F82530F582E4347FF583E0FF741C2576
:101F900030F582E4347DF583E06F60037F00220535
:101FA00030E530B406DAE4F53074142530F582E417
:101FB000347DF583E0FF74982530F582E43460F5D4
:101FC00083EFF00530E530B404DFE4F5307410251C
:101FD00030F582E4347DF583E0FF747D2530F582B1
:101FE000E43460F583EFF00530E530B404DFE4F568
:101FF0002F7E7D7F0074F02FFFE43EFEED2410FD68
:10200000EC34FFFCED2FFDEC3EFCC3EF9DEE9C405D
:10201000030221F58F828E83E014604B24FE607AE8
:1020200024FD70030220D024D3700302212324FE58
:10203000601A14700302217E243770030221F51404
:1020400060030221D90FBF00010E80BE0FBF000147
:102050000E0FBF00010E0FEFAA0670010E14F582DD
:102060008A83E0F52F80A30FBF00010E0FBF000190
:102070000EE4F530E530C39404508F0FEFAA0670DC
:10208000010E14F5828A83E0FB74812530F582E429
:102090003460F583EBF0053080DA0FBF00010E0FDE
:1020A000BF00010EE4F530E530C394044003022084
:1020B0000A0FEFAA0670010E14F5828A83E0FB7402
:1020C0008B2530F582E43460F583EBF0053080D762
:1020D0000FBF00010E0FEFAA0670010E14F5828AE1
:1020E00083E0F531E4F5300FEFAA0670010E14F528
:1020F000828A83E0FB748F2530F582E43460F583B7
:10210000EBF00530E530B404DEE4F530E53124FCD5
:10211000FBE530C39B400302200A0FBF00010E0500
:102120003080E90FBF00010E0FEFAA0670010E14F8
:10213000F5828A83E0F5310FEFAA0670010E14F5DF
:10214000828A83E0906074F00FEFAA0670010E148B
:10215000F5828A83E0906075F00FEFAA0670010E99
:1021600014F5828A83E0906076F00FEFAA06700182
:102170000E14F5828A83E0906077F002200A0FBF88
:1021800000010E0FEFAA0670010E14F5828A83E09B
:10219000F5310FEFAA0670010E14F5828A83E090E4
:1021A0006098F00FEFAA0670010E14F5828A83E0A2
:1021B000906099F00FEFAA0670010E14F5828A83E1
:1021C000E090609AF00FEFAA0670010E14F5828A73
:1021D00083E090609BF002200A0FBF00010E0FEF1A
:1021E000AA0670010E14F5828A83E0F5312FFFE410
:1021F0003EFE02200AAF2F228F2F8C308D318A3283
:102200008B33C2A8E52F75F003A424F0FFE5F0346A
:10221000818F82F583E0F5347F027E001254B2E5AF
:102220002F75F00CA4FFAEF02440FDEE34808D82BB
:10223000F583E0F537A3E0F538EF2440FFEE348076
:10224000FE8F82F583A3A3E0F5398F828E83A3A34B
:10225000A3E0F53AE52F75F003A424E2FFE5F0349E
:10226000818F82F583E0F5347F027E001254B2E55F
:102270002F75F00CA4FFAEF02418FDEE34808D8293
:10228000F583E0F53BA3E0F53CEF2418FFEE348046
:10229000FE8F82F583A3A3E0F53D8F828E83A3A3F7
:1022A000A3E0F53ED2A8AF3EAE3DAD3CAC3BAB3A71
:1022B000AA39A938A837C31206AE4029AE3DAF3EB1
:1022C000AC39AD3AED9FFFEC9EFEE52F25E0246290
:1022D000F582E43460F583E0FCA3E0C39FF536ECBF
:1022E0009EF535802EAE3DAF3EC3E49FFFE49EFEDB
:1022F000AC39AD3AEF2DFFEE3CFEE52F25E0246230
:10230000F582E43460F583E0FCA3E0C39FF536EC8E
:102310009EF535E52F25E02462F582E43460F583EF
:10232000E0FEA3E0C39536E5356480F8EE6480985E
:10233000501CE4FDAF2F122447EF64064E60057E6B
:10234000FF7FFF227F017E0012530C022202E5363E
:102350004535701BFDAF2F122447EF64064E600514
:102360007EFF7FFF227F017E0012530C022202C3F8
:10237000E5369533E5359532500685353285363369
:10238000E52F25E02410F8E6FA08E6FBE52F25E026
:1023900025E0244AF582E43460F583E0FCA3E0FD07
:1023A000A3E0FEA3E0553AFFEE5539FEED5538ECBB
:1023B0005537EF2BFFEE3AFAA9077B01AB018532C7
:1023C00067853368AD31AC30AF2F123AB6E4252FB4
:1023D000FFE434808F82F583E030E512E4FDAF2F17
:1023E000122447EF64064E60E47EFF7FFF22AE3288
:1023F000E4FCFDE53A2533F53AE5393EF539ED35AE
:1024000038F538EC3537F537E52F75F00CA4244056
:10241000FFE5F03480FE8F82F583E537F0A3E538E1
:10242000F08F828E83A3A3E539F08F828E83A3A3DE
:10243000A3E53AF0E4252FFFE434808F82F583741E
:1024400020F0AE32AF33228F63ED14602714700397
:102450000225892402600302268AE56375F018A428
:1024600024A0FFE5F034808F82F583E0756400F5E9
:1024700065022690C2A8E56375F003A424F0FFE589
:10248000F034818F82F583E0F5727F027E00125472
:10249000B2E56375F00CA4FFAEF02440FDEE34808D
:1024A0008D82F583E0F56AA3E0F56BEF2440FFEE43
:1024B0003480FE8F82F583A3A3E0F56C8F828E8338
:1024C000A3A3A3E0F56DE56375F003A424E2FFE5A3
:1024D000F034818F82F583E0F5727F027E00125422
:1024E000B2E56375F00CA4FFAEF02418FDEE348065
:1024F0008D82F583E0F56EA3E0F56FEF2418FFEE13
:102500003480FE8F82F583A3A3E0F5708F828E83E3
:10251000A3A3A3E0F571D2A8AF71AE70AD6FAC6E9E
:10252000AB6DAA6CA96BA86AC31206AE402AAE7046
:10253000AF71AC6CAD6DED9FFFEC9EFEE56325E0E9
:102540002462F582E43460F583E0FCA3E0C39FF5E8
:1025500065EC9EF564022690AE70AF71C3E49FFFF8
:10256000E49EFEAC6CAD6DEF2DFFEE3CFEE5632509
:10257000E02462F582E43460F583E0FCA3E0C39FCD
:10258000F565EC9EF564022690C2A8E56375F0033C
:10259000A424E0FFE5F034818F82F583E0F5727FBB
:1025A000027E001254B2E56375F00CA4FFAEF02475
:1025B00010FDEE34808D82F583E0F56AA3E0F56BC3
:1025C000EF2410FFEE3480FE8F82F583A3A3E0F5A5
:1025D0006C8F828E83A3A3A3E0F56DE56375F00392
:1025E000A424E1FFE5F034818F82F583E0F5727F6A
:1025F000027E001254B2E56375F00CA4FFAEF02425
:1026000014FDEE34808D82F583E0F566A3E0F56776
:10261000EF2414FFEE3480FE8F82F583A3A3E0F550
:10262000688F828E83A3A3A3E0F569D2A8AF69AEB9
:1026300068AD67AC66AB6DAA6CA96BA86AC31206DD
:10264000AE7006F564F5658047AF69AE68AD67ACFE
:1026500066AB6DAA6CA96BA86AD31206AE4012AE27
:1026600068AF69AC6CAD6DED9FF565EC9EF564806F
:102670001FAE68AF69C3E49FFFE49EFEAC6CAD6D16
:10268000EF2DF565EE3CF564800674FFF564F565A5
:10269000AE64AF6522AB07907D007401F0A3F0A398
:1026A0007406F0E4A3F0906093E0FCA3E0FDA3E0E7
:1026B000FEA3E0FF907D041206DFE4907D08F0A306
:1026C000F0A37480F0A3E4F0A3F0A3F0A3F0A3F0D0
:1026D000A3F0A3F0A3F0A3F0A3F0A3F0A3F0A3F062
:1026E000A3F0A3F0A3F0A3F0907FF8E0907D1CF09E
:1026F000907FF9E0907D1DF0907FFAE0907D1EF0D4
:10270000907FFBE0907D1FF0907FFCE0907D20F0BB
:10271000907FFDE0907D21F07F067E00741C2FF5F8
:1027200082E4347DF583E4F00FBF00010EEF641006
:102730004E70E9E4FEFF742C2FF582E4347DF583BE
:10274000E4F00FBF00010EEF64404E70E9E4FEFFBD
:10275000746C2FF582E4347DF583E4F00FBF000143
:102760000EEF64804E70E9907DEC7463F0A3748288
:10277000F0A37453F0A37463F0A37435F0A3740151
:10278000F0A37403F0A3743DF0A37407F0A37401E5
:10279000F0907FF8E0FD907DF6F0907FF9E0FC90FE
:1027A0007DF7F0907FFAE0F9907DF8F0907FFBE004
:1027B000907DF9F0907FFCE0907DFAF0907FFDE055
:1027C000907DFBF0A37432F0A37404F090607DE080
:1027D000907DFEF090607EE0907DFFF090607FE065
:1027E000907E00F0906080E0907E01F0A37436F05F
:1027F000A37404F0906098E0907E04F0906099E0FB
:10280000907E05F090609AE0907E06F090609BE0EC
:10281000907E07F0A3740CF0A3F0A37449F0A3F02A
:10282000A3744DF0A37437F0A37431F0A314F0A394
:10283000EDF0A3ECF0A3E9F0907FFBE0907E13F0C5
:10284000907FFCE0907E14F0907FFDE0907E15F08C
:10285000A37437F0A37405F0A37401F0A37403F01C
:10286000A37406F0A3743AF0A304F0A374FFF07EFF
:10287000007F3274EC2FF582747D3EF583E4F00F17
:10288000BF00010EBE01ECBF38E99060A0E4F0A3E8
:102890007443F0E4FEFF7E04782974FFF608DEFC42
:1028A000AF037543027544247545007546007547AE
:1028B000299060A0E0F548A3E0F5497B017A7D7995
:1028C0000012412722E49060D1F0A3F090602FE045
:1028D0009060ACF090600AE09060AEF0E4FD7F02A2
:1028E000122447EF4E60057F02124E177F017E00D3
:1028F0001252E69060ACE06401600302299F906090
:102900001DE0FFA3E09060B3CFF0A3EFF0E4FF740D
:10291000192FF582E43460F583E0FE74AF2FF58261
:10292000E43460F583EEF00FBF04E4906017E0FA42
:10293000A3E0FB7566807D027F0212490A9060ABBE
:102940007401F0200A097BFF7A44790E1255047D48
:10295000027F021224478E268F27D3EF9400EE6465
:102960008094805003022AACD3E5279400E52664C6
:1029700080948840067526087527007C637D007565
:102980003D01753E60753FCD7540017541607542F2
:10299000D1AB27AA267F021208BD8E268F27229050
:1029A00060AEE0FF64016005EF6402703F200A0939
:1029B0007BFF7A447917125357906017E0FAA3E02F
:1029C000FB7566807D017F0212490AEFF460EA7FA1
:1029D0000212546D200A097BFF7A447923125504B0
:1029E0009060AB7401F0E49060ADF0229060BAE4C6
:1029F00075F001120572ABF0FA7566807D017F02F9
:102A000012490ABFFF18C39060BBE094FF9060BA00
:102A1000E094FF40D77407F0A374D0F080CE200A72
:102A20001A9060BBE024FFFF9060BAE034FFFE1212
:102A300054D67BFF7A4479261253577B017A60790A
:102A40001990601DE0F52CA3E0F52D7F021242B82D
:102A5000BFFF1C200A097BFF7A447933125504E436
:102A60009060ABF09060ADF07F0AFE1252E62290CB
:102A700060AB7401F09060ADF0C292906030F0C233
:102A8000AFE49060B6F09060A2F0A3F09060C1F067
:102A9000A3F09060A8F0A3F09060A6F0A3F0D2AFEE
:102AA000200A097BFF7A44793812550422AB07903B
:102AB0007D007401F0A3F0A37406F0E4A3F090602D
:102AC00093E0FCA3E0FDA3E0FEA3E0FF907D0412F1
:102AD00006DFE4907D08F0A3F0A3F0A3F090607D02
:102AE000E0907D0CF090607EE0907D0DF090607F36
:102AF000E0907D0EF0906080E0907D0FF0E4A3F018
:102B0000A3F0A3F0A3F0A3F0A3F0A3F0A3F0A3F02D
:102B1000A3F0A3F0A3F0907FF8E0907D1CF0907FED
:102B2000F9E0907D1DF0907FFAE0907D1EF0907F9F
:102B3000FBE0907D1FF0907FFCE0907D20F0907F87
:102B4000FDE0907D21F07F067E00741C2FF582E46D
:102B5000347DF583E4F00FBF00010EEF64104E707A
:102B6000E9E4FEFF742C2FF582E4347DF583E4F074
:102B70000FBF00010EEF64404E70E9E4FEFF746C7D
:102B80002FF582E4347DF583E4F00FBF00010EEFF2
:102B900064804E70E9907DEC7463F0A37482F0A3BE
:102BA0007453F0A37463F0A37435F0A37401F0A31D
:102BB0007404F0A3743DF0A37407F0A37401F090C3
:102BC0007FF8E0907DF6F0907FF9E0907DF7F0904F
:102BD0007FFAE0907DF8F0907FFBE0907DF9F09037
:102BE0007FFCE0907DFAF0907FFDE0907DFBF0A30C
:102BF0007432F0A37404F090607DE0907DFEF0905C
:102C0000607EE0907DFFF090607FE0907E00F0902D
:102C10006080E0907E01F0A37436F0A37404F0901D
:102C20006098E0907E04F0906099E0907E05F090CE
:102C3000609AE0907E06F090609BE0907E07F0A3A3
:102C400074FFF07E007F1D74EC2FF582747D3EF5DD
:102C500083E4F00FBF00010EBE01ECBF38E975350B
:102C6000FF7536FF7537FF7538FFAF037543027583
:102C7000442475450075460075473575480075490B
:102C8000437B017A7D7900124127228F388C398D60
:102C90003A8A3B8B3CC2A8E53875F003A424E0FFD8
:102CA000E5F034818F82F583E0F53D7F027E0012EE
:102CB00054B2E53875F00CA4FFAEF02410FDEE34EC
:102CC000808D82F583E0F540A3E0F541EF2410FF0D
:102CD000EE3480FE8F82F583A3A3E0F5428F828ECF
:102CE00083A3A3A3E0F543E53875F003A424E1FF33
:102CF000E5F034818F82F583E0F53D7F027E00129E
:102D000054B2E53875F00CA4FFAEF02414FDEE3497
:102D1000808D82F583E0F544A3E0F545EF2414FFB0
:102D2000EE3480FE8F82F583A3A3E0F5468F828E7A
:102D300083A3A3A3E0F547D2A8D3E53C9400E53BE9
:102D400094005004E4FEFF22AF47AE46AD45AC44CC
:102D5000AB43AA42A941A840C31206AE4012AE46F8
:102D6000AF47AC42AD43ED9FF53FEC9EF53E80177B
:102D7000AE46AF47C3E49FFFE49EFEAC42AD43EFD7
:102D80002DF53FEE3CF53EC3E53F953CE53E953BDA
:102D9000501CE4FDAF38122447EF64064E60057EF8
:102DA000FF7FFF227F017E0012530C022C95E53835
:102DB00025E02408F8E6FA08E6FBE53825E025E0FA
:102DC000243AF582E43460F583E0FCA3E0FDA3E05F
:102DD000FEA3E05547FFEE5546FEED5545EC554444
:102DE000EF2BFFEE3AFAA9077B01FCAD01853B5CB6
:102DF000853C5DAB3AAA39AF381239B7AE3BE4FC3B
:102E0000FDE547253CF547E5463EF546ED3545F5FC
:102E100045EC3544F544E53875F00CA42414FFE581
:102E2000F03480FE8F82F583E544F0A3E545F08F12
:102E3000828E83A3A3E546F08F828E83A3A3A3E5AE
:102E400047F0E42538FFE434808F82F5837440F046
:102E5000AE3BAF3C22E49060CDF0A3F0752601AF0D
:102E6000261251BE74032526F582E43460F583EF03
:102E7000F074032526F582E43460F583E0FF90606A
:102E8000CEE02FF09060CDE03400F00526E526D3AB
:102E9000942E40CB7F3E1251BE9060CFEFF07F3F2B
:102EA0001251BE9060D0EFF0FD9060CFE0FE7C004C
:102EB000E42DFFEC3E9060D1F0A3EFF090602EE0A7
:102EC000702E9060D1E0FEA3E0FF9060CDE06E70C8
:102ED00003A3E06F601A7DFF7F3B12512D7DFF7FC2
:102EE0003C12512D7DFF7F3D12512D12000080FEBE
:102EF000E4F526E526242FFF1251BE74322526F56F
:102F000082E43460F583EFF00526E526C39408409B
:102F1000E290601FE0F52764BB603FE527F4603A6C
:102F2000E52764FE6034E52764FD602EE52764FA3A
:102F30006028E52764F46022E52764E8601CE52743
:102F400064D06016E52764A060107527FEAD277F6A
:102F50001C12512D90601FE527F0906020E09060DA
:102F6000A5F0906021E09060AAF09060A5E0FF6479
:102F7000086012EF6407600D7D087F1D12512D90CF
:102F800060207408F09060AAE0D39402400CE4FD45
:102F90007F1E12512DE4906021F0906022E06006C7
:102FA000E0D39402400D7D017F1F12512D906022CD
:102FB0007401F090600BE0D394E0400CE4FD7F08D6
:102FC00012512DE490600BF090602CE0FFA3E09094
:102FD00060D3CFF0A3EFF09060D3E064047004A35B
:102FE000E0640460287D047F2912512D7D047F2A2E
:102FF00012512D7DFF7F3B12512D7DFF7F3C1251E1
:103000002D7DFF7F3D12512D12000080FE22AB0767
:10301000907D007401F0A3F0A37406F0E4A3F09097
:103020006093E0FCA3E0FDA3E0FEA3E0FF907D043D
:103030001206DFE4907D08F0A3F0A37480F0A3E40F
:10304000F0A3F0A3F0A3F0A3F0A3F0A3F0A3F0A3E8
:10305000F0A3F0A3F0A3F0A3F0A3F0A3F0A3F0A3D8
:10306000F0907FF8E0907D1CF0907FF9E0907D1D5E
:10307000F0907FFAE0907D1EF0907FFBE0907D1F46
:10308000F0907FFCE0907D20F0907FFDE0907D212E
:10309000F07F067E00741C2FF582E4347DF583E416
:1030A000F00FBF00010EEF64104E70E9E4FEFF74F4
:1030B0002C2FF582E4347DF583E4F00FBF00010E80
:1030C000EF64404E70E9E4FEFF746C2FF582E43447
:1030D0007DF583E4F00FBF00010EEF64804E70E9D0
:1030E000907DEC7463F0A37482F0A37453F0A37426
:1030F00063F0A37435F0A37401F0A3F0A37437F068
:10310000A37405F0A37401F0A37403F0A37406F094
:10311000A3743AF0A304F0A374FFF07E007F0F7451
:10312000EC2FF582747D3EF583E4F00FBF00010EB5
:10313000BE01ECBF38E99060A0E4F0A37443F0E472
:10314000FEFF7E04782974FFF608DEFCAF037543AA
:10315000027544247545007546007547299060A0A6
:10316000E0F548A3E0F5497B017A7D79001241271B
:10317000228F26C2A8EF75F003A424F1FFE5F034F6
:10318000818F82F583E0F5277F027E001254B2E53D
:103190002675F00CA4FFAEF02444FDEE34808D8241
:1031A000F583E0F528A3E0F529EF2444FFEE348011
:1031B000FE8F82F583A3A3E0F52A8F828E83A3A3DB
:1031C000A3E0F52B7F027E001254B2C3E52B9401DD
:1031D000F52BE52A9400F52AE5299400F529E52840
:1031E0009400F528E52675F00CA42444FFE5F0349E
:1031F00080FE8F82F583E528F0A3E529F08F828E8B
:1032000083A3A3E52AF08F828E83A3A3A3E52BF0EB
:103210007F027E001254B2E52675F003A424E2FF7B
:10322000E5F034818F82F583E0F5277F027E00127E
:1032300054B2E52675F00CA4FFAEF02418FDEE3470
:10324000808D82F583E0F52CA3E0F52DEF2418FFA7
:10325000EE3480FE8F82F583A3A3E0F52E8F828E5D
:1032600083A3A3A3E0F52F7F027E001254B2C3E52F
:103270002F9401F52FE52E9400F52EE52D9400F501
:103280002DE52C9400F52CE52675F00CA42418FFF0
:10329000E5F03480FE8F82F583E52CF0A3E52DF078
:1032A0008F828E83A3A3E52EF08F828E83A3A3A3A8
:1032B000E52FF0D2A87F027E001254B2E42526FF4B
:1032C000E434808F82F5837420F0228E2B8F2C7F44
:1032D00001E4F52EF52FC2AF9060A8F0A3F0906046
:1032E000A6F0A3F0D2AFD200F519F51AEF600EE503
:1032F0002CB51AF8E52BB519F3E4FF80EF90000028
:10330000E0F52D64576004E4FEFF22900001E0F533
:103310002D64696004E4FEFF22900002E0F52D6454
:103320007A6004E4FEFF22900003E0F52D646E60F5
:1033300004E4FEFF22900004E0F52D64656004E4DF
:10334000FEFF22900005E0F52D64746004E4FEFFAA
:1033500022E4F530F531E52C24F8FFE52B34FFFEAF
:10336000C3E5319FE5309E502174062531F582E496
:103370003530F583E0F52D252FF52FE4352EF52E8C
:103380000531E5317002053080CC74FE252CF582C4
:1033900074FF352BF583E0F52DE52E652D600D7B53
:1033A000FF7A347932125357E4FEFF2274FF252C42
:1033B000F58274FF352BF583E0F52D652F600D7BCD
:1033C000FF7A347946125357E4FEFF22E4F519F5EB
:1033D0001AF530F531E52C24F8FFE52B34FFFEC358
:1033E000E5319FE5309E502574062531F582E435A0
:1033F00030F583E0853182853083F0051AE51A7057
:103400000205190531E5317002053080C8C200AEF1
:1034100019AF1A220A0D000A0D5472616E736665A7
:103420007220436F6E6669672046696C6520210AC9
:103430000D000A0D436865636B73756D20457272EC
:103440006F72203120000A0D436865636B73756DE0
:10345000204572726F722032000A0D46696C652039
:1034600073697A65203E3E20000A0D5472616E73C6
:103470006665722046696C6520210A0D000A0D44BC
:103480006F776E6C6F6164204572726F720A000A0A
:103490000D3E57616974202E20000A0D3E20436FB7
:1034A0006E666967000A0D3C693E203A20446973E4
:1034B000706C617920436F6E666967000A0D3C731A
:1034C0003E203A205265636569766520436F6E66DB
:1034D0006967000A0D3C633E203A204669726D77A9
:1034E00061726520557064617465000A0D3C643E2C
:1034F000203A2044697361626C652044484350005F
:103500000A0D3C773E203A20457261736520506178
:1035100073737764000A0D3C653E203A2045786954
:1035200074000A0D3E5479706520636F6D6D616E95
:1035300064203A20003E20000A0D49494D2056657E
:1035400072203A205354440A0D000001000A00641E
:1035500003E827109080007480F0E4F529E5292421
:1035600010FF748B2529F582E43460F583E0FD12A9
:10357000512D0529E529C3940440E27B017A607945
:103580008B12526EE4F529E529240CFF748125295C
:10359000F582E43460F583E0FD12512D0529E5291B
:1035A000C3940440E27B017A607981125246E4F5CB
:1035B00029E5292408FF747D2529F582E43460F586
:1035C00083E0FD12512D0529E529C3940440E27BD7
:1035D000017A60797D1252967B017A7F79F81252D6
:1035E000BE9080947403F07D557F5512107F300A91
:1035F00003023684752D01752E60752FCD7B017AFF
:103600006079981241F37BFF7A4F79E91253577B27
:10361000017A6079CD125504752D01752E60752FD4
:10362000CD7B017A60797D1241F37BFF7A4F79F986
:103630001253577B017A6079CD125504752D0175AF
:103640002E60752FCD7B017A6079811241F37BFF6B
:103650007A5079001253577B017A6079CD12550464
:10366000752D01752E60752FCD7B017A60798B12D7
:1036700041F37BFF7A5079071253577B017A6079C7
:10368000CD12550422C0E0C083C08263A201C08372
:10369000C082C0D075D000C004C005C006C007C23B
:1036A000AF209803023783300018AF99051AE51A46
:1036B000AC197002051914F5828C83EFF0C29802E0
:1036C00037839060A5E0B40719E599547FFF9060B7
:1036D000A8E0FCA3E02400F582746B3CF583EFF0D6
:1036E00080139060A8E0FEA3E02400F582746B3E96
:1036F000F583E599F09060A2E4F0A3F0906024E0F7
:10370000602B9060A8E0FEA3E0FF2400F582746BBC
:103710003EF583E0FD906024E0FCEDB5040FD20B94
:10372000EF2401FFE43E9060C3F0A3EFF09060232C
:10373000E0B4011F9060A8E0FEA3E02400F58274CD
:103740006B3EF583E0FFB41103751B00EFB4130368
:10375000751B019060A9E004F070069060A8E00479
:10376000F0C39060A8E094084004E4F0A3F09060F7
:1037700027E07002A3E06009D2019060C9E4F0A3E1
:10378000F0C298309904D203C299D2AFD007D006C4
:10379000D005D004D0D0D082D08363A201D082D013
:1037A00083D0E032752801124F0BE52870030238F0
:1037B000B29060A6E0FEA3E0FF9060A8E06E700308
:1037C000A3E06F60E59060A6E475F001120572FE5B
:1037D000740025F0F582746B3EF583E0F527FF1247
:1037E00050C67F0A1250C67F0D1250C6E527249D91
:1037F000604014604A1470030238A624F470030277
:10380000388B24FE602324FC605B240E60030238A6
:10381000AC12537A7F0A1250C67F0D1250C67BFF3E
:103820007A35793512535780811249ABE4F5280275
:1038300037AA124EBDEF4E60030237AAFEFF22E404
:10384000FD7F2B12512D7DFF7F3B12512D7DFF7F80
:103850003C12512D7DFF7F3D12512DE490602EF0E2
:10386000F5280237AA7DFF7F2E12512D7DFF7F3B69
:1038700012512D7DFF7F3C12512D7DFF7F3D125156
:103880002DE4906031F0F5280237AA7DFF7F3B12CE
:10389000512D7DFF7F3C12512D7DFF7F3D12512D1B
:1038A000E4F5280237AAE4F5280237AAE4F528024D
:1038B00037AA22906085E0C3940A400302396B90D6
:1038C000609CE0FCA3E0FDA3E0FEA3E0FF90608726
:1038D000E0F8A3E0F9A3E0FAA3E0FBC31206AE40D0
:1038E000030239B690609C1206EB00000000906065
:1038F0009CE0FCA3E0FDA3E0FEA3E02405FFE43E82
:10390000FEE43DFDE43CFC9060871206DF9060859C
:10391000E004F0906078E024FE601124FE6013243F
:103920000360030239B67F0112300E227F01122696
:1039300095227566807B447A007D027F0112490AD8
:10394000906093E0FCA3E0FDA3E0FEA3E0FFE4FAB7
:10395000F9F8EF2401FFEA3EFEE93DFDE83CFC906A
:1039600060931206DF7F0112269522200A097BFF51
:103970007A4F79DE1255049060977401F090609C44
:103980001206EB0000000090609CE0FCA3E0FDA3A9
:10399000E0FEA3E02405FFE43EFEE43DFDE43CFC44
:1039A0009060871206DFE4906085F07F0112300E90
:1039B0009060787401F0228F578C588D598A5A8BF9
:1039C0005BE55D455C7003FEFF22E4E55725E025DD
:1039D000E0243AF582E43460F583E0F8A3E0F9A34B
:1039E000E0FAA3E05559FBEA5558FAE4EB255DFBF4
:1039F000EA355CFAE433F9E433F8E55725E0245A74
:103A0000F582E43460F583E0FEA3E0FFEE3395E059
:103A1000FDFCD31206AE5003023A9EE4E55725E0C2
:103A200025E0243AF582E43460F583E0F8A3E0F978
:103A3000A3E0FAA3E05559FFEA5558FEE4E55725FF
:103A4000E0245AF582E43460F583E0FCA3E0C39FF0
:103A5000F55FEC9EF55EFEAF5FAA58A9597B01A801
:103A60005BAC5A7D0112080EC3E55D955FFFE55C16
:103A7000955EFEE55725E02408F8E6FC08E68C583C
:103A8000F559E55F255BF55BE55E355AF55AAA0405
:103A9000A9597B01A85BFC7D0112080E8013AE5C66
:103AA000AF5DAA58A9597B01A85BAC5A7D011208E9
:103AB0000EAE5CAF5D228F628C638D648A658B660F
:103AC000E56845677003FEFF22E4E56225E025E036
:103AD000244AF582E43460F583E0F8A3E0F9A3E03A
:103AE000FAA3E05566FBEA5565FAE4EB2568FBEAC4
:103AF0003567FAE433F9E433F8E56225E02462F54A
:103B000082E43460F583E0FEA3E0FFEE3395E0FD50
:103B1000FCD31206AE5003023B9BE4E56225E02590
:103B2000E0244AF582E43460F583E0F8A3E0F9A3E9
:103B3000E0FAA3E05566FFEA5565FEE4E56225E09C
:103B40002462F582E43460F583E0FCA3E0C39FF5D2
:103B50006AEC9EF569FEAF6AAA63A9647B01A86658
:103B6000AC657D0112080EC3E568956AFFE56795AF
:103B700069FEE56225E02410F8E6FC08E68C65F5B0
:103B800066E56A2564F564E5693563F563FAA96459
:103B90007B01A8667D0112080E8013AE67AF68AA8C
:103BA00063A9647B01A866AC657D0112080EAE674F
:103BB000AF6822C0E0C0F0C083C08263A201C083AE
:103BC000C082C0D075D000C000C006C007C2AFC25E
:103BD0008E7499258BF58B74F1258DF58D9060BDD4
:103BE000E004F070069060BCE004F0906027E070A4
:103BF00002A3E06028200C253001229060C9E47502
:103C0000F001120572FED3906028E095F0906027D5
:103C1000E09E5009D20C9060C9E4F0A3F0D390600C
:103C2000BDE094E89060BCE094034064E4F0A3F04D
:103C30009060ADE0B40130906029E07002A3E060D4
:103C4000269060A2E475F001120572FED390602AFE
:103C5000E095F0906029E09E500D9060B67401F000
:103C60009060A2E4F0A3F090602FE06401600C90FB
:103C7000600AE064016004E0B402159060BEE0FFF9
:103C800004F0EFD394B44008E4F0C2AFD202D2AF54
:103C9000D28ED2AFD007D006D000D0D0D082D08381
:103CA00063A201D082D083D0F0D0E0328F268C275F
:103CB0008D28E49060D1F0A3F0C2AF9060B6F09090
:103CC00060A2F0A3F09060C1F0A3F0D2AF90602F9B
:103CD000E064017036D3E52894F8E52794074006A0
:103CE0007527077528F87C637D00753D01753E607A
:103CF000753FCD7540017541607542D1AB28AA274B
:103D00007F021208BD8E278F288022D3E5289400D9
:103D1000E527940840067527087528007C637D0018
:103D2000AB28AA27AF26122C8B8E278F28D3E52805
:103D30009400E52794004065906023E0B4020A53A4
:103D400090BF7F647E001254B2E4F529F52AC3E5E2
:103D50002A9528E52995275033906023E0B4020680
:103D600012549EEF70FA7400252AF5827463352987
:103D7000F583E0FF1250C6906023E0B40104E51B18
:103D800070FC052AE52A7002052980C2906023E0B4
:103D9000B4020A7F907E011254B2439040228F6792
:103DA0007568008F6990606EE0FCA3E0FDA3E0FE03
:103DB000A3E0FFE4FAF9F8EF2401FFEA3EFEE93D53
:103DC000FDE83CFC90606E1206DF90606EE0FDE561
:103DD0006775F00CA42440FFE5F03480FE8F82F577
:103DE00083EDF090606FE08F828E83A3F09060701F
:103DF000E08F828E83A3A3F0906071E08F828E8328
:103E0000A3A3A3F07F027E001254B290606EE0FD87
:103E1000E56775F00CA42444FFE5F03480FE8F8242
:103E2000F583EDF090606FE08F828E83A3F0906059
:103E300070E08F828E83A3A3F0906071E08F828EFA
:103E400083A3A3A3F07F027E001254B290606EE0C1
:103E5000FDE56775F00CA42418FFE5F03480FE8FB3
:103E600082F583EDF090606FE08F828E83A3F090F7
:103E70006070E08F828E83A3A3F0906071E08F82E8
:103E80008E83A3A3A3F0227566807B447A007D0213
:103E90007F0112490A90607DE0F529A3E0F52AA38D
:103EA000E0F52BA3E0F52C75430075440A75450039
:103EB0007546007547297548137549887B007A0057
:103EC00079297F01124127EFF47002EEF4700302AA
:103ED0003F6B906086E004F07566807B447A007DDD
:103EE000027F0112490A7F01122AAD7F647E00120F
:103EF00052E6E4F533F534AF34124E170534E534A9
:103F000070020533C39404E533940040EA7F647E75
:103F1000001252E69080007480F0E4F533F534AF7F
:103F200034747D2FF582E43460F583E4F074292F36
:103F3000F8E4F60534E53470020533640445337063
:103F4000DE7B007A0079291252967B017A7F79F81C
:103F50001252BE7D557F5512107F7566807B447A64
:103F6000007D027F0112490A7F00227F0122124A4E
:103F7000E5EF6037D208300A030240497BFF7A43FD
:103F8000797B125357906074E0FCA3E0FDA3E0FE40
:103F9000A3E0FF1253DF7BFF7A4379901255047B35
:103FA000FF7A437991125357024049C208200A0907
:103FB0007BFF7A4379A1125357752608E4FDAF269B
:103FC00012512D74032526F582E43460F583E4F064
:103FD0000526E526D3941340E3125057200A097BA7
:103FE000FF7A4379B01253577566807BB47A057DAA
:103FF00002E4FF12490A7566807BB57A057D017F70
:104000000312490A7F0312546D752664AF261526E4
:10401000EF601C12443BBF010512443B80FB7F054F
:104020007E001252E6200AE47F2E1250C680DD7D0B
:10403000FF7F3B12512D7DFF7F3C12512D7DFF7F75
:104040003D12512D12000080FEA20822E4F533F546
:104050003478357C00FD7BFF7A35794AFE7F0A1281
:10406000080E753F01C2AFE49060A8F0A3F0906025
:10407000A6F0A3F0D2AFF52BF52CE53F606F906072
:10408000A6E0FEA3E0FFC39060A9E09FFF9060A8B8
:10409000E09EFED3EF9400EE940040DE9060A6E434
:1040A00075F001120572FE740025F0F582746B3E06
:1040B000F583E0F540FF1250C6E540B40D147F0AC9
:1040C0001250C6AF2B052B742D2FF876FFE4F53F69
:1040D0008011E54024D0FFAE2B052B742D2EF8A6C1
:1040E00007052CE52B64067091F53F808DE4F52BD8
:1040F000742D252BF8E6FFF460287E00152CE52CA6
:1041000025E02435F8E6FC08E6FD12052AEF253403
:10411000F534EE3533F533E52C6007052BE52BB48C
:1041200005CEAE33AF34228F3F8B408A418942D3D4
:10413000E5449400E54394005004E4FEFF22E54981
:104140004548601AE548FDE53F75F018A424ACFF2A
:10415000E5F034808F82F583EDF0E549A3F0AB45BF
:10416000AA46A9471204B0FDE53F75F018A424A89B
:10417000FFE5F03480FE8F82F583EDF090000112B0
:1041800004C98F828E83A3F09000021204C98F822B
:104190008E83A3A3F09000031204C98F828E83A3A1
:1041A000A3A3F0E4F54AF54BAB40E542254BF9E516
:1041B00041354AFA854350854451AF3F1213C5AD8E
:1041C00007AC06BCFF08BDFF057EFF7FFF22C3E5ED
:1041D000449DF544E5439CF543ED254BF54BEC350B
:1041E0004AF54AD3E5449400E543940050BAAE4AF8
:1041F000AF4B228B2A8A2B892CE4F530AB2AAA2BD1
:10420000A92CAF30EF3395E08F82F5831204C97586
:104210003100F532753100AE31FF7C007D6412054E
:104220003C12518FAB2D052FE52FAA2E7002052EC3
:1042300014F9EF1204F6AE31AF327C007D0A12059C
:104240003C7C007D0A12053CAF0512518FAB2D0559
:104250002FE52FAA2E7002052E14F9EF1204F6AEE8
:1042600031AF327C007D0A12053CAF0512518F122E
:10427000518FAB2D052FE52FAA2E7002052E14F9B4
:10428000EF1204F6AB2D052FE52FAA2E7002052E96
:1042900014F9742E1204F60530C3E530648094845A
:1042A00050030241FCAB2DE52F152F7002152E1483
:1042B000F9AA2EE41204F6228F28E52D452C602F52
:1042C000E52CFDE52875F018A424ACFFE5F034805A
:1042D0008F82F583EDF0E52DFDE52875F018A42417
:1042E000ACFFE5F034808F82F583A3EDF080037F8F
:1042F000FF221204B0FDE52875F018A424A8FFE5FC
:10430000F03480FE8F82F583EDF09000011204C935
:104310008F828E83A3F09000021204C98F828E8355
:10432000A3A3F09000031204C98F828E83A3A3A3DA
:10433000F0746A2528F582E43460F583E4F02528DA
:10434000FFE434808F82F5837404F0746A2528F5C5
:1043500082E43460F583E0700DFDAF28122447EF4E
:104360004E70E87FFF22746A2528F582E43460F5F8
:1043700083E020E2037FFF227F01223E2044484366
:1043800050206C656173652074696D65203D200067
:10439000003E204448435020537563636573732E79
:1043A000000A0D3E2044484350204661696C2E00AF
:1043B0000A0D3E2057616974000A0D49494D373195
:1043C0003030284129205665722E20342E34000AC0
:1043D0000D3E20436F6E66696720736F636B657473
:1043E000203A20004F4B2E2E003E20436F6E6E650C
:1043F00063746564003E20446973636F6E6E656329
:1044000074000A0D20524553544152542000554423
:1044100050206D6F6465003E204C697374656E209A
:104420003A20004F6B003E20636F6E6E6563742010
:104430003A20004661696C004F4B007D02E4FF1298
:1044400024478E278F28D3EF9400EE648094804019
:1044500030D3E52894F8E5276480948740067527D3
:10446000077528F8AD28AC27E4FF120CAB8F29E5BF
:1044700029B4020D12465F7F02124E17120000800F
:10448000FEE4FD7F03122447EF605524F9604A04DF
:1044900070617D027F031224478E278F28D3EF940B
:1044A00000EE64809480404BD3E5289400E52764B7
:1044B0008094884006752708752800AD28AC277FB2
:1044C00003120CAB8F29E5296402702712465F7F27
:1044D00002124E1712000080FE7F03124E17801347
:1044E0007566807BB57A057D017F0312490A7F03DB
:1044F00012546DAF29227529017BFF7A3579381264
:104500005357C2AFE49060A8F0A3F0D2AFE52960A2
:1045100020D39060A9E094009060A8E0940040ED62
:10452000906B00E0B453E67F521250C6E4F5298048
:10453000DCC2AFE49060A8F0A3F0D2AF752901E52A
:104540002960109060A8E07004A3E0645E70F0F54C
:104550002980ECE4F526F52774002527F582E4345C
:104560006BF583E0FF74012527F582E4346BF58356
:10457000E0FD12541A8F2805270527AD28AF261213
:10458000512D0526E526D3942E40CD7F431250C6EB
:104590007DFF7F3B12512D7DFF7F3C12512D7DFF12
:1045A0007F3D12512D12000080FE22C0E0C0F0C0FD
:1045B00083C08263A201C083C082C0D075D000C016
:1045C00000C001C002C004C005C006C007C2AFC21F
:1045D0008C74F1258AF58A74B1258CF58C300531FF
:1045E0009060B7E004F0E0B45027E4F090609CE005
:1045F000FCA3E0FDA3E0FEA3E0FFE4FAF9F8EF245A
:1046000001FFEA3EFEE93DFDE83CFC90609C12069D
:10461000DF9060ADE0B401239060C2E004F070066A
:104620009060C1E004F0D39060C2E094B39060C1A8
:10463000E094154006E4F0A3F0D206D28CD2AFD0BD
:1046400007D006D005D004D002D001D000D0D0D001
:1046500082D08363A201D082D083D0F0D0E03290A8
:104660007FF8E0FF907B04E06F600302470A907FD1
:10467000F9E0FF907B05E06F600302470A907FFA44
:10468000E0FF907B06E06F600302470A907FFBE04B
:10469000FF907B07E06F7072907FFCE0FF907B08DB
:1046A000E06F7066907FFDE0FF907B09E06F705ACD
:1046B000907B31E0B40120752A077403252AF58226
:1046C000E43460F583E0FDAF2A12512D052AE52A76
:1046D000D3943640E5801E752A077403252AF58297
:1046E000E43460F583E0FDAF2A12512D052AE52A56
:1046F000D3942E40E57DFF7F3B12512D7DFF7F3C03
:1047000012512D7DFF7F3D12512D43900422C0E0B8
:10471000C083C08263A201C083C082C0D075D000B4
:10472000C007C2A8908008E0FFEF607630E00E90EE
:104730008004E090606AF09080087401F0EF30E14E
:104740000E908005E090606BF09080087402F0EFAE
:1047500030E20E908006E090606CF0908008740467
:10476000F0EF30E30E908007E090606DF0908008ED
:104770007408F0EF30E4069080087410F0EF30E534
:10478000069080087420F0EF30E6069080087440B0
:10479000F0EF30E7069080087480F0908008E0FF2A
:1047A000808790800874FFF0D2A8D007D0D0D08244
:1047B000D08363A201D082D083D0E0328E268F27AF
:1047C000D3E5279400E526940050030248669060E4
:1047D00023E0B4010BAD27AC26AF1812515E8F1841
:1047E00090602FE0B4012685264385274475450156
:1047F0007546607547AF9060B3E0F548A3E0F549B2
:104800007B017A7379007F02124127800D7C737DD2
:1048100000AB27AA267F02124C549060A7E0252700
:10482000F09060A6E03526F0C3E09408400CA3E0C9
:104830002400F09060A6E034F8F0C2AFE49060C1CC
:10484000F0A3F0D2AF906027E07002A3E070069072
:104850006024E06011C2AFC20BC20CE49060C9F0EA
:10486000A3F0C201D2AF228D26C2ADE4F5C9D2CDEC
:10487000D2CCC2C9C2CAF5CDF5CCEF12071C48DDB7
:10488000A0489DBB48D5D048CDE848C5F448BDFAFE
:1048900048B5FD48ADFE48A5FF000048E37527FF79
:1048A0007528FA803E7527FF7528F480367527FF36
:1048B0007528E8802E7527FF7528DC80267527FF70
:1048C0007528B8801E7527FF75287080167527FE1D
:1048D0007528E0800E7527FD7528C080067527FBBA
:1048E0007528808527CB8528CA8527CD8528CCE5E6
:1048F00026B401057598508008E526B40303759821
:10490000D0D2CAE59924FF92CA228F62E5664DFD96
:10491000EF75F018A424A1FFE5F034808F82F583B1
:10492000EDF0EB4A601BEAF9E56275F018A424AEDD
:10493000FFE5F034808F82F583E9F0EBF9A3F08096
:1049400032906073E004F07006906072E004F090C2
:104950006072E0A3FDE56275F018A424AEFFE5F0F7
:104960003480FE8F82F583EDF0906073E08F828E4D
:1049700083A3F0746A2562F582E43460F583E4F081
:104980002562FFE434808F82F5837402F0746A2517
:1049900062F582E43460F583E0FF60F1EF20E1032B
:1049A0007FFF22AF62123D9EAF6222752C017BFF1A
:1049B0007A347917125357C2AFE49060A8F0A3F08D
:1049C0009060A6F0A3F0D2AFF52AE52C602A9060A3
:1049D000A8E07004A3E0645E7004F52C80EC052A66
:1049E0007F147E001252E67F2E1250C6E52AD39421
:1049F0000A40D712000080FEE4F529F52A7400254C
:104A00002AF582E4346BF583E0FF7401252AF582F0
:104A1000E4346BF583E0FD12541A8F2B052A052A26
:104A2000AD2BAF2912512D0529E529D3942E40CD68
:104A30007DFF7F3B12512D7DFF7F3C12512D7DFF6D
:104A40007F3D12512D12000080FE2278FFE4F6D83F
:104A5000FD9000007F007E80E4F0A3DFFCDEFA75AD
:104A60008172024AA0020026E493A3F8E493A340D3
:104A700003F68001F208DFF48029E493A3F85407D9
:104A8000240CC8C333C4540F4420C8834004F456D4
:104A9000800146F6DFE4800B01020408102040800C
:104AA000904F9BE47E019360BCA3FF543F30E50927
:104AB000541FFEE493A360010ECF54C025E060A80C
:104AC00040B8E493A3FAE493A3F8E493A3C8C5829F
:104AD000C8CAC583CAF0A3C8C582C8CAC583CADF0D
:104AE000E9DEE780BE200A097BFF7A50790E125575
:104AF000049060931206EB123456787566807B44FE
:104B00007A007D027F0112490A7F0112300E906007
:104B1000787401F0E4906086F090609C1206EB00DF
:104B200000000090609CE0FCA3E0FDA3E0FEA3E099
:104B30002405FFE43EFEE43DFDE43CFC906087126A
:104B400006DFE4906085F0D205906078E064036051
:104B5000191219FA906086E0C3940240037F002284
:104B6000906097E0B401E27F00227F0122E4FF120F
:104B700051BE8F267F011251BE8F277F021251BE78
:104B80008F287F031251BE8F29E526B4AA0FE5278F
:104B9000700BE528B40806E52964DC604AE4FF12DE
:104BA000521A8F267F0112521A8F277F0212521A31
:104BB0008F287F0312521A8F29E52664AA7028E5F0
:104BC000277024E528B4081FE529B4DC1AE4F52A87
:104BD000AF2A12521A8F2BAD2BAF2A12512D052A54
:104BE000E52AC3944040E9227F3B1251BE8F27E55E
:104BF0002764AA605E7F3C1251BE8F27E52764556B
:104C000060517F3D1251BE8F27E52764AA6044E4BE
:104C1000F528F529752601AF261251BEEF2529F595
:104C200029E43528F5280526E526D3942E40E87D8D
:104C3000AA7F3B12512D7D557F3C12512D7DAA7FBD
:104C40003D12512DE528FD7F3E12512DAD297F3FAC
:104C500012512D228F288C298D2A8A2B8B2CD3E55B
:104C60002C9400E52B94005004E4FEFF22E4F52D83
:104C7000F52EE52A252EFDE529352DFCAB2CAA2B9A
:104C8000AF281221F8AD07AC06BCFF08BDFF057EBA
:104C9000FF7FFF22C3E52C9DF52CE52B9CF52BED2A
:104CA000252EF52EEC352DF52DD3E52C9400E52B96
:104CB000940050BEAE2DAF2E22E4F5267F027E007A
:104CC0001252E6D39060A9E094009060A8E09400AE
:104CD00040329060A6E475F001120572FE74002562
:104CE000F0F582746B3EF583E0B470189060A6E036
:104CF000FEA3E02400F582746B3EF583E0FF1250C2
:104D0000C61237A47F2E1250C60526E526C3940787
:104D100040AA22C200E49060A8F0A3F09060A6F040
:104D2000A3F0F518F51B9060B6F09060A2F0A3F028
:104D300090609C1206EB00000000C208E49060C185
:104D4000F0A3F0C2069060BCF0A3F0C20BC20C90BE
:104D500060C9F0A3F09060B7F0C2099060ABF0A317
:104D6000F0A3F0D292906030F0223E20436F6E6646
:104D700069674D73672072656365697665000A0D22
:104D80003E576169742E003E446F776E6C6F6164AC
:104D9000204572726F72000A0D3E4E65742D55707B
:104DA0006772616465000A0D3E43616E63656C0A5B
:104DB0000D000A0D3E436865636B73756D203A20E4
:104DC000008F3AE53AC4540FFFC3940A400FEF75C1
:104DD000F00A84E5F02441FF1250C68011E53AC480
:104DE000540F75F00A84E5F02430FF1250C6E53AFE
:104DF000540FFFC3940A400EEF75F00A84E5F024C7
:104E000041FF1250C622E53A540F75F00A84E5F0CE
:104E10002430FF1250C6228F62E4FD122447EF4E69
:104E200060487D01AF62122447E56225E02462F507
:104E300082E43460F583E0FCA3E06F7002EC6E70F6
:104E400029746A2562F582E43460F583E4F0256212
:104E5000FFE434808F82F5837410F0746A2562F564
:104E600082E43460F583E030E3F122E4FD9060A554
:104E7000E0FCB408047E808006ECB407027E40E4C7
:104E8000FC9060A5E014FBECD39B5011EFA8040844
:104E90008002C333D8FC5E60010D0C80E49060AAF0
:104EA000E0FCB4020AED30E0037F01227F0022EC37
:104EB000B40109ED20E0037F01227F00227BFF7A0D
:104EC00034795912535712404C8E298F2A7BFF7A1E
:104ED000347969125357AF2AAE291232CBEF4E7094
:104EE0000D7BFF7A34797D125357E4FEFF227BFF5E
:104EF0007A34798F125357E52A24F8907FFFF0E532
:104F00002934FF907FFEF012501B227BFF7A347908
:104F10009A1253577BFF7A3479A51253577BFF7A45
:104F20003479BC1253577BFF7A3479D31253577BB1
:104F3000FF7A3479EB1253577BFF7A35790012539D
:104F4000577BFF7A3579151253577BFF7A357922D3
:104F500012535722C0E0C083C08263A201C083C045
:104F600082C0D075D000C006C007C2AA300202C2FB
:104F7000029060A6E0FEA3E0FFA3E06E7003A3E052
:104F80006F6002D209D2AAD007D006D0D0D082D08A
:104F90008363A201D082D083D0E0324260A60000B9
:104FA0004260A800004260C900004260A2000041C7
:104FB00060B6004260C300004260C100004160B7BB
:104FC00000011800011B00C10BC10CC101C1094146
:104FD00060BE00C1024160850041609700000A0D7B
:104FE00054696D65204F7574002044484350205328
:104FF0006572766572203A2000204950203A2000E0
:1050000020534D203A2000204757203A20000A0D17
:105010003E44484350206D6F646500C2AFE4F539EB
:10502000F53AE4253AFFE539345D8F82F583E49360
:10503000F538E4253AFFE5393470FEAD3812539D5A
:10504000053AE53A70020539C39454E539940240B3
:10505000D112700080FE221254527B017A7F79F8BF
:105060001252BEE4FF7F047827E4F608DFFC7B00E1
:105070007A00792712526E7B007A00792712524605
:105080007B007A0079271252967D557F5512107F4A
:10509000221254527B017A7F79F81252BE7B017A38
:1050A00060791312526E7B017A60790F1252467B3F
:1050B000017A60790B1252969080947403F07D55BA
:1050C0007F5512107F22AA07E4F99060AAE06022BF
:1050D000124E6BA9079060A5E0FFB40708E96012C3
:1050E000430280800DEFB40809E96004D29B80027E
:1050F000C29B3003FD8A99C203228F2FC2AFE4F90D
:105100005390FDE52FA801088002C333D8FC30E797
:105110000543900180035390FE7F017E001253BF30
:1051200043900209B908D95390FDD2AF228F2D8D3B
:105130002EC2931255127FA01250FA1254F5E52D8B
:105140002480FF1250FA1254F5AF2E1250FA125466
:10515000F512551F7F0A7E001253BFD293228C286E
:105160008D29EF7017D3E5299400E5289404401E9B
:10517000C2AF7F131250C6D2AF7F0122C3E528947D
:1051800002500BC2AF7F111250C6D2AF7F0022AEC9
:1051900007C3EE64809480400DD3EE648094895000
:1051A00005EE2430FF22C3EE6480948A400DD3EED6
:1051B0006480948F5005EE2437FF22AF06228F2C97
:1051C000D2931255127FA01250FA1254F5E52C24F6
:1051D00080FF1250FA1254F51255127FA11250FAA4
:1051E0001254F51251ED12552C12551F22E4FFC234
:1051F000AF5390FD7E07439002E59030E00D7401BF
:10520000A806088002C333D8FC42075390FD1EC392
:10521000EE6480948050DFD2AF228F2CD29312554F
:10522000127FA01250FA1254F5AF2C1250FA1254F9
:10523000F51255127FA11250FA1254F51251ED12C7
:10524000552C12551F228B388A39893AE4FFAB3826
:10525000AA39A93A8F827583001204C9FE74842F7B
:10526000F582E43480F583EEF00FBF04E1228B3841
:105270008A39893AE4FFAB38AA39A93A8F82758313
:10528000001204C9FE74802FF582E43480F583EEA9
:10529000F00FBF04E1228B388A39893AE4FFAB383A
:1052A000AA39A93A8F827583001204C9FE748E2F21
:1052B000F582E43480F583EEF00FBF04E1228B38F1
:1052C0008A39893AE4FFAB38AA39A93A8F827583C3
:1052D000001204C9FE74882FF582E43480F583EE51
:1052E000F00FBF06E1228E388F39E4F53AF53BC363
:1052F000E53B9539E53A953850117F0A7E00125307
:105300000C053BE53B7002053A80E4228E628F6318
:10531000E4F564F565C3E5659563E5649562501150
:105320007FE87E031254B20565E56570020564806E
:10533000E422C2AFC28CC28E758900438911758A7E
:10534000F1758CB1758B99758DF1C2B9D2A9D2ABBB
:10535000D28CD28ED2AF228B388A39893AE4F53B8F
:10536000AB38AA39A93A853B827583001204C9FF7C
:1053700060071250C6053B80E7227BFF7A34791420
:10538000125357752901AF291251BE124DC17F200A
:105390001250C60529E529D3942E40EA228D3BA25E
:1053A000AF920DC2AF8E838F8274021254C4E53B5C
:1053B00043A2201254C653A2DFA20D92AFFF22E4F3
:1053C000FDFCC3ED9FEC9E5015E4FBFA0BBB000106
:1053D0000ABA03F8BBE8F50DBD00010C80E4228F8A
:1053E0002A8E298D288C27E4FBFA7901F812060E03
:1053F0001254D6E52AFFE529FEE41254D62274D0D1
:105400002FFFD364809489400474F92FFFD3EF6495
:1054100080948F400474E02FFF228F2D8D2E125325
:10542000FE8F2DE52DC454F0F52DAF2E1253FEEF57
:10543000252DF52DFF22E4F5267F037E0012530C67
:10544000E59020E2031237A40526E526C394034025
:10545000E8229060727403F0A374E8F090606E121A
:1054600006EB122334459080007480F022746A2F7A
:10547000F582E43460F583E4F02FFFE434808F821A
:10548000F5837408F022E4FF1251BEBFFF0F7D01C7
:105490007FFE1248671254E6D2AF1244F622C2AF22
:1054A000E590FED2AF30E7037F0122EE20E7027FD6
:1054B0000022E4FDFCC3ED9FEC9E50070DBD0001F2
:1054C0000C80F222F922C002C004C00612FFF0D004
:1054D00006D004D002228E388F39E538FF124DC134
:1054E000AF39124DC12275B81075B710D203C298EA
:1054F000C299D2AC225390FD439002E5905408FF2C
:105500005390FD221253577F0A1250C67F0D12503E
:10551000C6224390014390025390FE5390FD2253C4
:1055200090FD5390FE439002439001225390FD431F
:1055300090014390025390FD22C288D2A8C2AA22B1
:10554000000000000000000000000000000000005B
:10555000000000000000000000000000000000004B
:10556000000000000000000000000000000000003B
:10557000000000000000000000000000000000002B
:105D0000027240C2AF7F281271828F10907FFEE036
:105D1000F50CA3E0F50DE4F50EF50FF50AF50BF51E
:105D200008F509E50CC4F854F0C868FEE50DC45444
:105D30000F48FFC3E5099FE5089E5049AE0EAF0F1F
:105D4000AD07AC067B10AF0BAE0A12711F741025A5
:105D50000FF50FE4350EF50E7410250BF50BE43539
:105D60000AF50AE5107014AE08AF097C017DF41243
:105D700070CAED4C70057F2312724C0509E509705D
:105D8000A20508809EE50CC4F854F0C868FEE50D35
:105D9000C4540F48C4F8540FC868FFEEC454F04808
:105DA000FEC3E50D9FFFE50C9EAC0EAD0FAB07AF3C
:105DB0000BAE0A12711F53A2DFE4F5F0F5D0758126
:105DC00007F582F58312000080FEBC000BBE00299F
:105DD000EF8DF084FFADF022E4CCF875F008EF2FE2
:105DE000FFEE33FEEC33FCEE9DEC984005FCEE9D9F
:105DF000FE0FD5F0E9E4CEFD22EDF8F5F0EE8420BB
:105E0000D21CFEADF075F008EF2FFFED33FD40071B
:105E1000985006D5F0F222C398FD0FD5F0EA228BF8
:105E200011A2AF9200C2AF85A21253A2FE8E838F41
:105E30008205A28C838D8274091271F8E51153A238
:105E4000FE43A2201271FA53A2DF8512A2A2009291
:105E5000AFFF228F12E4F95390FDE512A8010880EC
:105E600002C333D8FC30E70543900180035390FE12
:105E70007F017E001271D843900209B908D953906E
:105E8000FD228F111272197FA012715312720AE54E
:105E9000112480FF12715312720A1272197FA1121B
:105EA000715312720A1271AF12723312722622E407
:105EB000FF5390FD7E07439002E59030E00D7401A2
:105EC000A806088002C333D8FC42075390FD1EC3C6
:105ED000EE6480948050DF22E4FDFCC3ED9FEC9ED5
:105EE0005015E4FBFA0BBB00010ABA03F8BBE8F556
:105EF0000DBD00010C80E422F922C002C004C006DE
:105F000012FFF0D006D004D002225390FD4390023D
:105F1000E5905408FF5390FD2243900143900253B3
:105F200090FE5390FD225390FD5390FE4390024308
:105F30009001225390FD4390014390025390FD2223
:105F400078FFE4F6D8FD7581200270038F993099AF
:045F5000FDC29922D3
:00000001FF
